:020000040000FA
:040800002BEF09F0E1
:1008100003B26DEF05F0F2B48BEF05F09EB093EFED
:1008200005F09EB29BEF05F0F2A81AEF04F0F2B2C9
:100830001CEF04F0DAEF08F0CD90F2929EA026EFC4
:1008400004F00101533F26EF04F0542BAEC1B2F186
:10085000AFC1B3F1B0C1B4F1B1C1B5F1AAC1AEF14C
:10086000ABC1AFF1ACC1B0F1ADC1B1F1A6C1AAF15C
:10087000A7C1ABF1A8C1ACF1A9C1ADF1A2C1A6F16C
:10088000A3C1A7F1A4C1A8F1A5C1A9F19EC1A2F17C
:100890009FC1A3F1A0C1A4F1A1C1A5F19AC19EF18C
:1008A0009BC19FF19CC1A0F19DC1A1F196C19AF19C
:1008B00097C19BF198C19CF199C19DF1CECF96F162
:1008C000CFCF97F153C198F154C199F1CF6ACE6A55
:1008D0000101536B546B9E90CD800FBC0F8E0FBAED
:1008E00075EF04F00F8ADAEF08F00F8C0FBEB1EF4E
:1008F00004F096C19AF197C19BF198C19CF199C1FE
:100900009DF19AC19EF19BC19FF19CC1A0F19DC137
:10091000A1F19EC1A2F19FC1A3F1A0C1A4F1A1C107
:10092000A5F1A2C1A6F1A3C1A7F1A4C1A8F1A5C1D7
:10093000A9F1A6C1AAF1A7C1ABF1A8C1ACF1A9C1A7
:10094000ADF1AAC1AEF1ABC1AFF1ACC1B0F1ADC177
:10095000B1F1AEC1B2F1AFC1B3F1B0C1B4F1B1C147
:10096000B5F101015E6B5F6B606B616B96515E2749
:1009700097515F2398516023995161239A515E27C3
:100980009B515F239C5160239D5161239E515E27A3
:100990009F515F23A0516023A1516123A2515E2783
:1009A000A3515F23A4516023A5516123A6515E2763
:1009B000A7515F23A8516023A9516123AA515E2743
:1009C000AB515F23AC516023AD516123AE515E2723
:1009D000AF515F23B0516023B1516123B2515E2703
:1009E000B3515F23B4516023B5516123D890010105
:1009F000613360335F335E33D8900101613360331C
:100A00005F335E33D8900101613360335F335E330F
:100A100000C10CF101C10DF102C10EF103C10FF1D2
:100A200004C110F105C111F106C112F107C113F1A2
:100A300008C114F109C115F10AC116F10BC117F172
:100A400034C135F111B830EF05F00101620E046FC9
:100A5000010E056F000E066F000E076F39EF05F0EF
:100A60000101A70E046F020E056F000E066F000E47
:100A7000076F5EC100F15FC101F160C102F161C1A8
:100A800003F105EC1FF003BF04D019BE02D019A07A
:100A9000108C11A051EF05F010BA51EF05F00F8046
:100AA000108A0CC100F10DC101F10EC102F10FC19C
:100AB00003F110C104F111C105F112C106F113C116
:100AC00007F114C108F115C109F116C10AF117C1E6
:100AD0000BF135C134F1DAEF08F00392ABB2AB9809
:100AE000AB88030103EE00F080517F0BE92604C0C0
:100AF000EFFF802B8151805D700BD8A48B820000AA
:100B00008051815D700BD8A48B9281518019D8B42B
:100B10000790DAEF08F0F2940101453FDAEF08F0B0
:100B2000462BDAEF08F09E900101533FDAEF08F010
:100B3000542BDAEF08F09E9211B80AEF07F08BB44D
:100B4000A9EF05F010ACA9EF05F08B84109CAAEF7B
:100B500005F08B94C3CF55F1C4CF56F1C28207B4D0
:100B600014EF06F047C14BF148C14CF149C14DF1BA
:100B70004AC14EF15EC162F15FC163F160C164F1CF
:100B800061C165F196C1B6F197C1B7F198C1B8F1ED
:100B900099C1B9F19AC1BAF19BC1BBF19CC1BCF139
:100BA0009DC1BDF19EC1BEF19FC1BFF1A0C1C0F109
:100BB000A1C1C1F1A2C1C2F1A3C1C3F1A4C1C4F1D9
:100BC000A5C1C5F1A6C1C6F1A7C1C7F1A8C1C8F1A9
:100BD000A9C1C9F1AAC1CAF1ABC1CBF1ACC1CCF179
:100BE000ADC1CDF1AEC1CEF1AFC1CFF1B0C1D0F149
:100BF000B1C1D1F1B2C1D2F1B3C1D3F1B4C1D4F119
:100C0000B5C1D5F1010155515B2756515C23E86A06
:100C10005D230E2E14EF06F05CC157F15DC158F153
:100C20005B6B5C6B5D6B078E0201002FDAEF08F0E7
:100C30003C0E006F1A50E00BE00AE866128818BEFE
:100C400002D018B4108E00C10CF101C10DF102C127
:100C50000EF103C10FF104C110F105C111F106C17C
:100C600012F107C113F108C114F109C115F10AC14C
:100C700016F10BC117F134C135F101018A6748EF54
:100C800006F08B6748EF06F08C6748EF06F08D673B
:100C90004CEF06F07CEF06F08EC100F18FC101F140
:100CA00090C102F191C103F10101010E046F000E28
:100CB000056F000E066F000E076F05EC1FF000C1F8
:100CC0008EF101C18FF102C190F103C191F1006772
:100CD00071EF06F0016771EF06F0026771EF06F041
:100CE00003677CEF06F08AC18EF18BC18FF18CC156
:100CF00090F18DC191F10F80D57ED5BE6DD0D6CF4C
:100D000047F1D7CF48F145C149F1E86AE8CF4AF148
:100D100019BE02D019A0108C109047C100F148C133
:100D200001F149C102F14AC103F101010A0E046F48
:100D3000000E056F000E066F000E076F05EC1FF02A
:100D400003AF1080010154A7B2EF06F00F9A0F9C79
:100D50000F9E0101000E5E6F600E5F6F3D0E606FB3
:100D6000080E616F010147BFC2EF06F04867C2EF8E
:100D700006F04967C2EF06F04A67C2EF06F0F28854
:100D8000E7EF06F0F2985E6B5F6B606B616B966BE2
:100D9000976B986B996B9A6B9B6B9C6B9D6B9E6B27
:100DA0009F6BA06BA16BA26BA36BA46BA56BA66BD7
:100DB000A76BA86BA96BAA6BAB6BAC6BAD6BAE6B87
:100DC000AF6BB06BB16BB26BB36BB46BB56BD76A17
:100DD000D66A0101456B466B0CC100F10DC101F1F2
:100DE0000EC102F10FC103F110C104F111C105F1EF
:100DF00012C106F113C107F114C108F115C109F1BF
:100E000016C10AF117C10BF135C134F1DAEF08F060
:100E1000DAEF08F00201002F63EF08F0D59ED6CF7D
:100E200047F1D7CF48F145C149F1E86AE8CF4AF127
:100E3000D76AD66A0101456B466BD58E1A50E00B16
:100E4000E00AE866128818BE02D018B4108E17AEF9
:100E50001C8C00C10CF101C10DF102C10EF103C1E6
:100E60000FF104C110F105C111F106C112F107C162
:100E700013F108C114F109C115F10AC116F10BC132
:100E800017F134C135F10FA0109A11B853EF07F0E4
:100E90000101620E046F010E056F000E066F000E59
:100EA000076F5CEF07F00101A70E046F020E056FDC
:100EB000000E066F000E076F47C100F148C101F137
:100EC00049C102F14AC103F105EC1FF003BF6FEF06
:100ED00007F019BE02D019A0108C11B00F800CC100
:100EE00000F10DC101F10EC102F10FC103F110C1FA
:100EF00004F111C105F112C106F113C107F114C1CA
:100F000008F115C109F116C10AF117C10BF135C17C
:100F100034F102013C0E006F00C10CF101C10DF172
:100F200002C10EF103C10FF104C110F105C111F1AD
:100F300006C112F107C113F108C114F109C115F17D
:100F40000AC116F10BC117F134C135F101018A67ED
:100F5000B1EF07F08B67B1EF07F08C67B1EF07F0E7
:100F60008D67B5EF07F0E5EF07F08EC100F18FC197
:100F700001F190C102F191C103F10101010E046F71
:100F8000000E056F000E066F000E076F05EC1FF0D8
:100F900000C18EF101C18FF102C190F103C191F145
:100FA0000067DAEF07F00167DAEF07F00267DAEFC0
:100FB00007F00367E5EF07F08AC18EF18BC18FF16F
:100FC0008CC190F18DC191F10F80109047C100F15B
:100FD00048C101F149C102F14AC103F101010A0E00
:100FE000046F000E056F000E066F000E076F05EC14
:100FF0001FF003AF1080010154A70BEF08F00F9A08
:101000000F9C0F9E0101000E5E6F600E5F6F3D0E24
:10101000606F080E616F47C100F148C101F149C11D
:1010200002F14AC103F10101140E046F050E056FB0
:10103000000E066F000E076F05EC1FF003AF24EFE4
:1010400008F0F28849EF08F0F2985E6B5F6B606B16
:10105000616B966B976B986B996B9A6B9B6B9C6BA8
:101060009D6B9E6B9F6BA06BA16BA26BA36BA46B24
:10107000A56BA66BA76BA86BA96BAA6BAB6BAC6BD4
:10108000AD6BAE6BAF6BB06BB16BB26BB36BB46B84
:10109000B56B0CC100F10DC101F10EC102F10FC120
:1010A00003F110C104F111C105F112C106F113C120
:1010B00007F114C108F115C109F116C10AF117C1F0
:1010C0000BF135C134F18BB46DEF08F010AC6DEF5E
:1010D00008F08B84109C6EEF08F08B94C3CF55F111
:1010E000C4CF56F1C28207B4D8EF08F047C14BF124
:1010F00048C14CF149C14DF14AC14EF15EC162F1A6
:101100005FC163F160C164F161C165F196C1B6F17F
:1011100097C1B7F198C1B8F199C1B9F19AC1BAF1C3
:101120009BC1BBF19CC1BCF19DC1BDF19EC1BEF193
:101130009FC1BFF1A0C1C0F1A1C1C1F1A2C1C2F163
:10114000A3C1C3F1A4C1C4F1A5C1C5F1A6C1C6F133
:10115000A7C1C7F1A8C1C8F1A9C1C9F1AAC1CAF103
:10116000ABC1CBF1ACC1CCF1ADC1CDF1AEC1CEF1D3
:10117000AFC1CFF1B0C1D0F1B1C1D1F1B2C1D2F1A3
:10118000B3C1D3F1B4C1D4F1B5C1D5F10101555109
:101190005B2756515C23E86A5D230E2ED8EF08F0DA
:1011A0005CC157F15DC158F15B6B5C6B5D6B078E89
:1011B000DAEF08F002C0E0FF005001C0D8FF1000D5
:1011C000A6B2E0EF08F00CC0A9FF0BC0A8FFA69ED6
:1011D000A69CA684F29E550EA76EAA0EA76EA682A6
:1011E000F28EA694A6B2F2EF08F00C2A1200A96EB5
:1011F000A69EA69CA680A8500C2A120004012C0EC4
:10120000826F29EC0BF000EC20F00C50F7EC08F0AA
:10121000E8CF00F10C50F7EC08F0E8CF01F101AF96
:1012200017EF09F00101FF0E026FFF0E036FA3EC31
:101230001FF0296723EF09F00401200E826F29ECCB
:101240000BF028EF09F004012D0E826F29EC0BF052
:10125000CDEC1DF01200076A0F6A106A116A126A5B
:10126000136A0F010E0EC16E860EC06E030EC26EA3
:101270000F01896A190E926E080E8A6EF10E936E36
:101280008B6A980E946EF18EFC0EF7EC08F0E8CFA6
:101290000BF00BA011800BA211820BA411840BA8E0
:1012A0001188C90EF7EC08F0E8CF17F0CA0EF7EC7A
:1012B00008F0E8CF18F0CB0EF7EC08F0E8CF19F003
:1012C000CC0EF7EC08F0E8CF1AF0CD0EF7EC08F0F2
:1012D000E8CF2FF01C6A1D6A0E6A01015B6B5C6B24
:1012E0005D6B576B586BF29A0101476B486B496B0A
:1012F0004A6B4B6B4C6B4D6B4E6B4F6B506B516B2A
:10130000526B456B466BD76AD66A0F01280ED56EB5
:10131000F28A9D90B00ECD6E01015E6B5F6B606BCB
:10132000616B626B636B646B656B666B676B686B41
:10133000696B536B546BCF6ACE6A0F9A0F9C0F9EEA
:101340009D80760ECA6E9D8202013C0E006FCC6AB3
:10135000160EF7EC08F0E8CF00F1170EF7EC08F0E6
:10136000E8CF01F1180EF7EC08F0E8CF02F1190E02
:10137000F7EC08F0E8CF03F1010103AFDAEF09F071
:1013800000EC20F0160E0C6E00C10BF0E0EC08F043
:10139000170E0C6E01C10BF0E0EC08F0180E0C6E8D
:1013A00002C10BF0E0EC08F0190E0C6E03C10BF05B
:1013B000E0EC08F000C18AF101C18BF102C18CF1AF
:1013C00003C18DF100C18EF101C18FF102C190F115
:1013D00003C191F11A0EF7EC08F0E8CF00F11B0EF3
:1013E000F7EC08F0E8CF01F11C0EF7EC08F0E8CFBD
:1013F00002F11D0EF7EC08F0E8CF03F1010103AF95
:1014000030EF0AF000EC20F01A0E0C6E00C10BF069
:10141000E0EC08F01B0E0C6E01C10BF0E0EC08F0E4
:101420001C0E0C6E02C10BF0E0EC08F01D0E0C6EF1
:1014300003C10BF0E0EC08F01A0EF7EC08F0E8CF6F
:1014400000F11B0EF7EC08F0E8CF01F11C0EF7ECF1
:1014500008F0E8CF02F11D0EF7EC08F0E8CF03F139
:1014600000C192F101C193F102C194F103C195F160
:10147000240EAC6E900EAB6E240EAC6E080EB86EE1
:1014800080B661EF0AF01E0EF7EC08F0E8CF00F12D
:101490001F0EF7EC08F0E8CF01F100C1E8FFFF0AEA
:1014A00010E001C1E8FFFF0A0CE01E0EF7EC08F0A7
:1014B000E8CFAFFF1F0EF7EC08F0E8CFB0FF65EF05
:1014C0000AF0000EB06E1F0EAF6E0401806B816BD0
:1014D0000F01900EAB6E0F019D8A0301806B816B33
:1014E000C26B8B9207900001F28EF28C07B07BEFFB
:1014F0001CF00FB017EF16F010BE17EF16F012B871
:1015000017EF16F00301805181197F0BD8B47BEFE0
:101510001CF013EE00F081517F0BE126812BE7CF09
:10152000E8FFE00BD8B47BEF1CF023EE82F0C25151
:101530003F0BD926E7CFDFFFC22BDF50780AD8A4B4
:101540007BEF1CF007808EC100F18FC101F190C1CB
:1015500002F191C103F10101040E046F000E056F49
:10156000000E066F000E076F05EC1FF000AFC2EF14
:101570000AF00101030E8E6F000E8F6F000E906F48
:10158000000E916F03018251720AD8B4FCEF15F07E
:101590008251520AD8B4FCEF15F08251750AD8B4C2
:1015A000FCEF15F08251630AD8B435EF19F082517F
:1015B000690AD8B4ABEF12F082517A0AD8B4BEEF00
:1015C00013F08251490AD8B44AEF12F08251500AFE
:1015D000D8B468EF11F08251700AD8B4ABEF11F0B3
:1015E0008251540AD8B4D6EF11F08251740AD8B49B
:1015F0001CEF12F08251410AD8B43FEF0CF0825137
:101600004B0AD8B43DEF0BF082516D0AD8B472EF9B
:1016100010F082514D0AD8B48BEF10F08251730A4A
:10162000D8B42CEF15F08251530AD8B491EF15F0CD
:101630008251620AD8B41AEF11F08251420AD8B42A
:1016400055EF11F08251590AD8B4C3EF0FF06CEF87
:1016500019F0040114EE00F080517F0BE12682C4E2
:10166000E7FF802B120004010D0E826F29EC0BF0B6
:101670000A0E826F29EC0BF0120004014B0E826FF0
:1016800029EC0BF004012C0E826F29EC0BF081B8D1
:1016900002D02FB630D003018351430AD8B482EF71
:1016A0000BF003018351630AD8B484EF0BF00301FC
:1016B0008351520AD8B486EF0BF003018351720AAA
:1016C000D8B488EF0BF003018351470AD8B48AEFEE
:1016D0000BF003018351670AD8B48CEF0BF00301C0
:1016E0008351540AD8B48EEF0BF003018351740A6E
:1016F000D8B4FDEF0BF003018351550AD8B490EF35
:101700000BF082D02F807AD02F9078D02F8276D095
:101710002F9274D02F8472D02F9470D02F866ED0D9
:1017200084C330F185C331F186C332F187C333F10D
:101730000101296B4EEC20F0C5EC1FF000C104F153
:1017400001C105F102C106F103C107F141EC20F02E
:10175000200EF86EF76AF66A0900F5CF2CF1090041
:10176000F5CF2DF10900F5CF2EF10900F5CF2FF1BE
:101770000900F5CF30F10900F5CF31F10900F5CFBF
:1017800032F10900F5CF33F10101296B4EEC20F065
:10179000C5EC1FF005EC1FF00067D6EF0BF00167FA
:1017A000D6EF0BF00267D6EF0BF0036701D025D020
:1017B00004014E0E826F29EC0BF004016F0E826F54
:1017C00029EC0BF004014D0E826F29EC0BF00401A3
:1017D000610E826F29EC0BF00401740E826F29EC0C
:1017E0000BF00401630E826F29EC0BF00401680E0C
:1017F000826F29EC0BF06AEF19F02F96CD0E0C6E6C
:101800002FC00BF0E0EC08F0CD0EF7EC08F0E8CFBD
:101810002FF02FB006D00401630E826F29EC0BF07D
:1018200005D00401430E826F29EC0BF02FB206D0D5
:101830000401720E826F29EC0BF005D00401520EE8
:10184000826F29EC0BF02FB406D00401670E826F73
:1018500029EC0BF005D00401470E826F29EC0BF048
:101860002FB606D00401740E826F29EC0BF005D060
:101870000401540E826F29EC0BF06AEF19F0040199
:10188000410E826F29EC0BF003018351310AD8B469
:10189000E3EF0EF003018351320AD8B413EF0EF0D8
:1018A00003018351330AD8B49CEF0DF00301835137
:1018B000340AD8B48CEF0CF003018351350AD8B444
:1018C00069EF0CF004013F0E826F29EC0BF06AEF18
:1018D00019F004012C0E826F29EC0BF003018451E6
:1018E000300AD8B47CEF0CF003018451310AD8B42B
:1018F00084EF0CF0D5EF0DF08B900401300E826F69
:1019000029EC0BF08AEF0CF08B800401310E826F12
:1019100029EC0BF06AEF19F0CC0EF7EC08F0E8CFE9
:101920000BF004012C0E826F29EC0BF003018451A3
:10193000310AD8B4B0EF0CF003018451300AD8B4A6
:10194000B2EF0CF0030184514D0AD8B4BCEF0CF097
:1019500003018451540AD8B4C3EF0CF0DAEF0CF051
:101960008A8401D08A940BAE04D00BAC02D00BBA9F
:1019700021D0E00E0B1218D01F0E0B168539E8444B
:10198000E00B0B1211D0E00E0B1641EC20F085C3DA
:1019900032F186C333F10101296B4EEC20F0C5EC26
:1019A0001FF000511F0B0B12CC0E0C6E0BC00BF076
:1019B000E0EC08F00401340E826F29EC0BF0040116
:1019C0002C0E826F29EC0BF0CC0EF7EC08F0E8CF70
:1019D0001AF08AB406D00401300E826F29EC0BF0A5
:1019E00005D00401310E826F29EC0BF004012C0E9E
:1019F000826F29EC0BF01A38E840070BE8CF82F42D
:101A00000401300E822729EC0BF004012C0E826FAA
:101A100029EC0BF000EC20F01A501F0BE8CF00F17E
:101A2000A3EC1FF032C182F40401300E822729ECAE
:101A30000BF033C182F40401300E822729EC0BF045
:101A400004012C0E826F29EC0BF000EC20F02DC06D
:101A500000F100AF0BD0FF0E016FFF0E026FFF0E03
:101A6000036F04012D0E826F29EC0BF0A3EC1FF025
:101A700031C182F40401300E822729EC0BF032C10F
:101A800082F40401300E822729EC0BF033C182F47A
:101A90000401300E822729EC0BF004012C0E826F1A
:101AA00029EC0BF000EC20F02CC000F1A3EC1FF0AF
:101AB00031C182F40401300E822729EC0BF032C1CF
:101AC00082F40401300E822729EC0BF033C182F43A
:101AD0000401300E822729EC0BF004012C0E826FDA
:101AE00029EC0BF000EC20F02EC000F100AF0BD081
:101AF000FF0E016FFF0E026FFF0E036F04012D0E2C
:101B0000826F29EC0BF0A3EC1FF031C182F40401C9
:101B1000300E822729EC0BF032C182F40401300E22
:101B2000822729EC0BF033C182F40401300E8227A6
:101B300029EC0BF06AEF19F0CB0EF7EC08F0E8CFC8
:101B40000BF004012C0E826F29EC0BF00301845181
:101B5000450AD8B4C0EF0DF003018451440AD8B44B
:101B6000C3EF0DF003018451300AD8B4C6EF0DF075
:101B700003018451310AD8B4CAEF0DF0D5EF0DF04E
:101B80000B9ECFEF0DF00B8ECFEF0DF0FC0E0B1672
:101B9000CFEF0DF0FC0E0B160B80CFEF0DF0CB0E40
:101BA0000C6E0BC00BF0E0EC08F00401330E826FFA
:101BB00029EC0BF004012C0E826F29EC0BF0CB0EFC
:101BC000F7EC08F0E8CF19F019BEEEEF0DF00401C4
:101BD000450E826F29EC0BF0F3EF0DF00401440E7B
:101BE000826F29EC0BF004012C0E826F29EC0BF0B4
:101BF0000401300E826F29EC0BF004012C0E826F71
:101C000029EC0BF019B00CEF0EF00401300E826FCE
:101C100029EC0BF011EF0EF00401310E826F29EC6C
:101C20000BF06AEF19F0CA0EF7EC08F0E8CF0BF0F2
:101C300004012C0E826F29EC0BF003018451450A3C
:101C4000D8B44FEF0EF003018451440AD8B452EFD8
:101C50000EF0030184514D0AD8B45BEF0EF003017E
:101C60008451410AD8B455EF0EF003018451460A5D
:101C7000D8B458EF0EF003018451560AD8B463EF7C
:101C80000EF003018451500AD8B46EEF0EF0030138
:101C90008451520AD8B471EF0EF07AEF0EF00B9E19
:101CA00074EF0EF00B8E74EF0EF00B9C74EF0EF0D1
:101CB0000B8C74EF0EF0FC0E0B1685C3E8FF030BC4
:101CC0000B1274EF0EF0C70E0B1685C3E8FF070B5F
:101CD000E846E846E8460B1274EF0EF00B8474EF0A
:101CE0000EF00B9474EF0EF0CA0E0C6E0BC00BF0DE
:101CF000E0EC08F0CA0EF7EC08F0E8CF18F00401A9
:101D0000320E826F29EC0BF004012C0E826F29EC4D
:101D10000BF018BE93EF0EF00401450E826F29EC14
:101D20000BF098EF0EF00401440E826F29EC0BF0DB
:101D300004012C0E826F29EC0BF018C0E8FF030B96
:101D4000E8CF82F40401300E822729EC0BF0040165
:101D50002C0E826F29EC0BF018BCB6EF0EF00401CC
:101D6000410E826F29EC0BF0BBEF0EF00401460E22
:101D7000826F29EC0BF004012C0E826F29EC0BF022
:101D800018C0E8FF380BE842E842E842E8CF82F4A6
:101D90000401300E822729EC0BF004012C0E826F17
:101DA00029EC0BF018B4DCEF0EF00401520E826F38
:101DB00029EC0BF0E1EF0EF00401500E826F29ECDC
:101DC0000BF06AEF19F0C90EF7EC08F0E8CF0BF052
:101DD00004012C0E826F29EC0BF003018451450A9B
:101DE000D8B401EF0FF003018451440AD8B404EFD2
:101DF0000FF0030184514D0AD8B407EF0FF015EF2F
:101E00000FF00B9E0FEF0FF00B8E0FEF0FF0F80E91
:101E10000B1685C3E8FF070B0B120FEF0FF0C90E6F
:101E20000C6E0BC00BF0E0EC08F00401310E826F79
:101E300029EC0BF004012C0E826F29EC0BF0C90E7B
:101E4000F7EC08F0E8CF17F017BE06D00401450EF6
:101E5000826F29EC0BF005D00401440E826F29EC4F
:101E60000BF004012C0E826F29EC0BF017C0E8FF79
:101E7000070BE8CF82F40401300E822729EC0BF027
:101E800004012C0E826F29EC0BF0078000EC20F08F
:101E900028C0E8FF003B00430043030BA3EC1FF006
:101EA00033C182F40401300E822729EC0BF00401C7
:101EB0002C0E826F29EC0BF000EC20F028C001F111
:101EC000019F019D29C000F10101A3EC1FF02FC16A
:101ED00082F40401300E822729EC0BF030C182F429
:101EE0000401300E822729EC0BF031C182F4040189
:101EF000300E822729EC0BF032C182F40401300E3F
:101F0000822729EC0BF033C182F40401300E8227C2
:101F100029EC0BF004012C0E826F29EC0BF000EC85
:101F200020F02AC001F12BC000F1D890013300331A
:101F3000D890013300330101A3EC1FF02FC182F4CC
:101F40000401300E822729EC0BF030C182F4040129
:101F5000300E822729EC0BF031C182F40401300EDF
:101F6000822729EC0BF032C182F40401300E822763
:101F700029EC0BF033C182F40401300E822729ECE6
:101F80000BF06AEF19F0FC0EF7EC08F0E8CF0BF05D
:101F900003018351520AD8B4FAEF0FF003018351C1
:101FA000720AD8B4FDEF0FF003018351500AD8B480
:101FB00000EF10F003018351700AD8B403EF10F062
:101FC00003018351550AD8B406EF10F00301835181
:101FD000750AD8B409EF10F003018351430AD8B44D
:101FE00012EF10F003018351630AD8B415EF10F01B
:101FF0001EEF10F00B9018EF10F00B8018EF10F0A0
:102000000B9218EF10F00B8218EF10F00B9418EFF2
:1020100010F00B8418EF10F00B9618EF10F00B86F1
:1020200018EF10F00B9818EF10F00B8818EF10F065
:10203000FC0E0C6E0BC00BF0E0EC08F00401590E26
:10204000826F29EC0BF01190119211941198FC0EF3
:10205000F7EC08F0E8CF0BF00BA011800BA2118277
:102060000BA411840BA8118811A03EEF10F00401FD
:10207000520E826F29EC0BF043EF10F00401720E48
:10208000826F29EC0BF011A84DEF10F00401430E04
:10209000826F29EC0BF052EF10F00401630E826F97
:1020A00029EC0BF011A25CEF10F00401500E826FCE
:1020B00029EC0BF061EF10F00401700E826F29EC37
:1020C0000BF011A46BEF10F00401550E826F29EC98
:1020D0000BF070EF10F00401750E826F29EC0BF01D
:1020E0006AEF19F004016D0E826F29EC0BF0030109
:1020F0008351300AD8B4CAEF10F003018351310A7A
:10210000D8B4DDEF10F003018351320AD8B4F0EFF8
:1021100010F06CEF19F004014D0E826F29EC0BF0FA
:1021200041EC20F084C331F185C332F186C333F131
:102130000101296B4EEC20F0C5EC1FF00301835127
:10214000300AD8B4B2EF10F003018351310AD8B489
:10215000BAEF10F003018351320AD8B4C2EF10F085
:102160006CEF19F0FD0E0C6E00C10BF0E0EC08F006
:10217000CAEF10F0FE0E0C6E00C10BF0E0EC08F0A0
:10218000DDEF10F0FF0E0C6E00C10BF0E0EC08F07C
:10219000F0EF10F00401300E826F29EC0BF0040117
:1021A0002C0E826F29EC0BF000EC20F0FD0EF7EC0A
:1021B00008F0E8CF00F101EF11F00401310E826F59
:1021C00029EC0BF004012C0E826F29EC0BF000ECD3
:1021D00020F0FE0EF7EC08F0E8CF00F101EF11F06F
:1021E0000401320E826F29EC0BF000EC20F00401A8
:1021F0002C0E826F29EC0BF0FF0EF7EC08F0E8CF05
:1022000000F1A3EC1FF031C182F40401300E8227EB
:1022100029EC0BF032C182F40401300E822729EC44
:102220000BF033C182F40401300E822729EC0BF04D
:102230006AEF19F08351610AD8A46CEF19F0845148
:10224000750AD8A46CEF19F08551640AD8A46CEF14
:1022500019F086C32AF187C32BF188C32CF189C3F7
:102260002DF18AC32EF18BC32FF18CC330F18DC3B6
:1022700031F18EC332F18FC333F10101296B4EEC82
:1022800020F0C5EC1FF000C1AFFF01C1B0FF1E0E72
:102290000C6EAFCF0BF0E0EC08F01F0E0C6EB0CF61
:1022A0000BF0E0EC08F06CEF19F080B65FEF11F086
:1022B0000401300E826F29EC0BF064EF11F0040181
:1022C000310E826F29EC0BF033EC0BF06CEF19F050
:1022D00083C32AF184C32BF185C32CF186C32DF16E
:1022E00087C32EF188C32FF189C330F18AC331F13E
:1022F0008BC332F18CC333F101014EEC20F0C5ECFD
:102300001FF0160E0C6E00C10BF0E0EC08F0170E7B
:102310000C6E01C10BF0E0EC08F0180E0C6E02C15F
:102320000BF0E0EC08F0190E0C6E03C10BF0E0ECC2
:1023300008F000C18AF101C18BF102C18CF103C127
:102340008DF100C18EF101C18FF102C190F103C185
:1023500091F14AEF12F083C32AF184C32BF185C3B4
:102360002CF186C32DF187C32EF188C32FF189C3C9
:1023700030F18AC331F18BC332F18CC333F10101E7
:102380004EEC20F0C5EC1FF000C18AF101C18BF1C9
:1023900002C18CF103C18DF100C18EF101C18FF139
:1023A00002C190F103C191F14AEF12F083C32AF107
:1023B00084C32BF185C32CF186C32DF187C32EF185
:1023C00088C32FF189C330F18AC331F18CC332F154
:1023D0008DC333F101014EEC20F0C5EC1FF001017B
:1023E000000E046F000E056F010E066F000E076FE2
:1023F00016EC1FF01A0E0C6E00C10BF0E0EC08F0AA
:102400001B0E0C6E01C10BF0E0EC08F01C0E0C6E04
:1024100002C10BF0E0EC08F01D0E0C6E03C10BF0D6
:10242000E0EC08F000C192F101C193F102C194F116
:1024300003C195F14AEF12F083C32AF184C32BF153
:1024400085C32CF186C32DF187C32EF188C32FF1EC
:1024500089C330F18AC331F18CC332F18DC333F1BA
:1024600001014EEC20F0C5EC1FF00101000E046FDD
:10247000000E056F010E066F000E076F16EC1FF0C1
:1024800000C192F101C193F102C194F103C195F130
:102490004AEF12F0160EF7EC08F0E8CF00F1170E35
:1024A000F7EC08F0E8CF01F1180EF7EC08F0E8CFF0
:1024B00002F1190EF7EC08F0E8CF03F1A3EC1FF0DE
:1024C00086EC1DF00401730E826F29EC0BF0040101
:1024D0002C0E826F29EC0BF08AC100F18BC101F147
:1024E0008CC102F18DC103F1A3EC1FF086EC1DF04D
:1024F0000401730E826F29EC0BF004012C0E826F25
:1025000029EC0BF01A0EF7EC08F0E8CF00F11B0EE7
:10251000F7EC08F0E8CF01F11C0EF7EC08F0E8CF7B
:1025200002F11D0EF7EC08F0E8CF03F187EC19F08B
:1025300004012C0E826F29EC0BF092C100F193C1C3
:1025400001F194C102F195C103F187EC19F033EC6C
:102550000BF06CEF19F00401690E826F29EC0BF09F
:1025600004012C0E826F29EC0BF00101040E006FA8
:10257000000E016F000E026F000E036FA3EC1FF040
:102580002CC182F40401300E822729EC0BF02DC1FE
:1025900082F40401300E822729EC0BF02EC182F464
:1025A0000401300E822729EC0BF02FC182F40401C4
:1025B000300E822729EC0BF030C182F40401300E7A
:1025C000822729EC0BF031C182F40401300E8227FE
:1025D00029EC0BF032C182F40401300E822729EC81
:1025E0000BF033C182F40401300E822729EC0BF08A
:1025F00004012C0E826F29EC0BF00101050E006F17
:10260000000E016F000E026F000E036FA3EC1FF0AF
:102610002CC182F40401300E822729EC0BF02DC16D
:1026200082F40401300E822729EC0BF02EC182F4D3
:102630000401300E822729EC0BF02FC182F4040133
:10264000300E822729EC0BF030C182F40401300EE9
:10265000822729EC0BF031C182F40401300E82276D
:1026600029EC0BF032C182F40401300E822729ECF0
:102670000BF033C182F40401300E822729EC0BF0F9
:1026800004012C0E826F29EC0BF00101300E006F5B
:10269000000E016F000E026F000E036FA3EC1FF01F
:1026A0002CC182F40401300E822729EC0BF02DC1DD
:1026B00082F40401300E822729EC0BF02EC182F443
:1026C0000401300E822729EC0BF02FC182F40401A3
:1026D000300E822729EC0BF030C182F40401300E59
:1026E000822729EC0BF031C182F40401300E8227DD
:1026F00029EC0BF032C182F40401300E822729EC60
:102700000BF033C182F40401300E822729EC0BF068
:1027100004012C0E826F29EC0BF0200EF86EF76A84
:10272000F66A04010900F5CF82F429EC0BF00900E8
:10273000F5CF82F429EC0BF00900F5CF82F429ECF7
:102740000BF00900F5CF82F429EC0BF00900F5CF6E
:1027500082F429EC0BF00900F5CF82F429EC0BF0A0
:102760000900F5CF82F429EC0BF00900F5CF82F4D3
:1027700029EC0BF033EC0BF06CEF19F08351630A8A
:10278000D8A46AEF19F08451610AD8A46AEF19F04D
:1027900085516C0AD8A46AEF19F08651410A3FE0CE
:1027A0008651440A1BE08651420AD8B422EF14F045
:1027B0008651350AD8B4F6EF1AF08651360AD8B4E5
:1027C0004BEF1BF08651370AD8B4B4EF1BF086519B
:1027D000380AD8B412EF1CF06AEF19F00798079A7C
:1027E00004017A0E826F29EC0BF00401780E826FDF
:1027F00029EC0BF00401640E826F29EC0BF004014C
:10280000550E826F29EC0BF00BEF14F004014C0E07
:10281000826F29EC0BF033EC0BF06CEF19F00788AA
:10282000079A04017A0E826F29EC0BF00401410E25
:10283000826F29EC0BF00401610E826F29EC0BF022
:10284000FFEF13F00798078A04017A0E826F29ECD4
:102850000BF00401420E826F29EC0BF00401610EB3
:10286000826F29EC0BF0FFEF13F00101666740EF78
:1028700014F0676740EF14F0686740EF14F0696781
:1028800015D04F674BEF14F050674BEF14F05167C2
:102890004BEF14F052670AD00101000E006F000EDA
:1028A000016F000E026F000E036F120011B80AD004
:1028B0000101620E046F010E056F000E066F000E1F
:1028C000076F09D00101A70E046F020E056F000EFD
:1028D000066F000E076F66C100F167C101F168C1A4
:1028E00002F169C103F105EC1FF003BFE8EF14F03A
:1028F000119A119C0101000E046FA80E056F550E70
:10290000066F020E076F66C100F167C101F168C171
:1029100002F169C103F166C186F167C187F168C13F
:1029200088F169C189F105EC1FF003BF0BD00101EB
:10293000000E866FA80E876F550E886F020E896F86
:10294000118A119C0E0EF7EC08F0E8CF18F10F0E6B
:10295000F7EC08F0E8CF19F1100EF7EC08F0E8CF2B
:102960001AF1110EF7EC08F0E8CF1BF14EEC1EF057
:1029700086C104F187C105F188C106F189C107F15B
:1029800005EC1FF0078212EC1EF04EEC1EF00792D1
:1029900012EC1EF086C100F187C101F188C102F17D
:1029A00089C103F1079212EC1EF0CC0E046FE00E09
:1029B000056F870E066F050E076F05EC1FF000C14F
:1029C00018F101C119F102C11AF103C11BF13BD089
:1029D000119C119A0101800E006F1A0E016F060EF4
:1029E000026F000E036F4FC104F150C105F151C1D8
:1029F00006F152C107F105EC1FF003AF05D000EC62
:102A000020F0118C119A12000E0EF7EC08F0E8CFAE
:102A100018F10F0EF7EC08F0E8CF19F1100EF7ECF3
:102A200008F0E8CF1AF1110EF7EC08F0E8CF1BF12F
:102A30004FC100F150C101F151C102F152C103F186
:102A4000078212EC1EF018C100F119C101F11AC180
:102A500002F11BC103F112000401730E826F29EC15
:102A60000BF004012C0E826F29EC0BF0078462C17D
:102A700066F163C167F164C168F165C169F14BC179
:102A80004FF14CC150F14DC151F14EC152F157C1FE
:102A900059F158C15AF1079452EC15F033EC0BF090
:102AA0006CEF19F066C100F167C101F168C102F174
:102AB00069C103F10101A3EC1FF086EC1DF00401D4
:102AC000630E826F29EC0BF004012C0E826F29EC4F
:102AD0000BF04FC100F150C101F151C102F152C1DF
:102AE00003F10101A3EC1FF086EC1DF00401660E5A
:102AF000826F29EC0BF004012C0E826F29EC0BF095
:102B000000EC20F059C100F15AC101F10101A3EC20
:102B10001FF086EC1DF00401740E826F29EC0BF09F
:102B2000120010820401530E826F29EC0BF0040195
:102B30002C0E826F29EC0BF083C32AF184C32BF196
:102B400085C32CF186C32DF187C32EF188C32FF1E5
:102B500089C330F18AC331F18BC332F18CC333F1B5
:102B600001014EEC20F0C5EC1FF000C166F101C17F
:102B700067F102C168F103C169F18EC32AF18FC305
:102B80002BF190C32CF191C32DF192C32EF193C37D
:102B90002FF194C330F195C331F196C332F197C34D
:102BA00033F101014EEC20F0C5EC1FF000C14FF1F4
:102BB00001C150F102C151F103C152F141EC20F0C9
:102BC00099C32FF19AC330F19BC331F19CC332F109
:102BD0009DC333F101014EEC20F0C5EC1FF000C1A4
:102BE00059F101C15AF152EC15F004012C0E826F1B
:102BF00029EC0BF00BEF16F0118E19A002D019AED4
:102C0000108C18BE02D018A4108E8251520A02E114
:102C10000F8201D00F928251750A02E1108401D017
:102C200010948251550A02E1108601D0109611A02D
:102C300003D011A401D01084078410B279EF16F0EC
:102C400010A465EF16F0B6C166F1B7C167F1B8C15F
:102C500068F1B9C169F1BAC16AF1BBC16BF1BCC11C
:102C60006CF1BDC16DF1BEC16EF1BFC16FF1C0C1EC
:102C700070F1C1C171F1C2C172F1C3C173F1C4C1BC
:102C800074F1C5C175F1C6C176F1C7C177F1C8C18C
:102C900078F1C9C179F1CAC17AF1CBC17BF1CCC15C
:102CA0007CF1CDC17DF1CEC17EF1CFC17FF1D0C12C
:102CB00080F1D1C181F1D2C182F1D3C183F1D4C1FC
:102CC00084F1D5C185F16DEF16F062C166F163C183
:102CD00067F164C168F165C169F14BC14FF14CC145
:102CE00050F14DC151F14EC152F157C159F158C186
:102CF0005AF107940FA09BEF16F00101926788EF3D
:102D000016F0936788EF16F0946788EF16F09567D2
:102D10008CEF16F09BEF16F035EC14F092C104F135
:102D200093C105F194C106F195C107F105EC1FF0BF
:102D300003BF32EF19F035EC14F00101000E046FFF
:102D4000000E056F010E066F000E076F36EC1FF0C8
:102D500011A02CD011A22AD0A3EC1FF0296701D01A
:102D600007D004012D0E826F29EC0BF030EF19F023
:102D700030C182F40401300E822729EC0BF031C1FE
:102D800082F40401300E822729EC0BF032C182F468
:102D90000401300E822729EC0BF033C182F40401C8
:102DA000300E822729EC0BF030EF19F012A8C5D0B5
:102DB00012981AC01BF01B3A1B42070E1B1600018B
:102DC0001B50000AD8B469EF17F000011B50010A2C
:102DD000D8B4F5EF16F000011B50020AD8B4F3EF97
:102DE00016F09BEF17F09BEF17F000EC20F02AC0D5
:102DF00001F12BC000F1D89001330033D89001339A
:102E000000330101630E046F000E056F000E066FA4
:102E1000000E076F36EC1FF0280E046F000E056FD2
:102E2000000E066F000E076F05EC1FF000C12DF0BD
:102E300000EC20F028C001F1019F019D29C000F1A4
:102E40000101A40E046F000E056F000E066F000E48
:102E5000076F36EC1FF000C12CF000C104F101C176
:102E600005F102C106F103C107F1640E006F000E07
:102E7000016F000E026F000E036F05EC1FF0050ED0
:102E8000046F000E056F000E066F000E076F36EC24
:102E90001FF000C104F101C105F102C106F103C137
:102EA00007F100EC20F02DC000F105EC1FF000C18F
:102EB0002EF02EC0E8FF050F2D5C03E78A849BEF00
:102EC00017F02EC0E8FF0A0F2D5C01E68A949BEFF5
:102ED00017F000C124F101C125F102C126F103C19F
:102EE00027F100EC20F006EC20F01A501F0BE8CF81
:102EF00000F10101640E046F000E056F000E066FF5
:102F0000000E076F16EC1FF024C104F125C105F176
:102F100026C106F127C107F105EC1FF003BF02D05F
:102F20008A9401D08A8424C100F125C101F126C10F
:102F300002F127C103F132EF19F000C124F101C100
:102F400025F102C126F103C127F110AE4CD0109E2D
:102F500000C108F101C109F102C10AF103C10BF17D
:102F6000A3EC1FF030C1D6F131C1D7F132C1D8F195
:102F700033C1D9F108C100F109C101F10AC102F15F
:102F80000BC103F101016C0E046F070E056F000EFB
:102F9000066F000E076F05EC1FF003BF04D00101A0
:102FA000550EDA6F1CD008C100F109C101F10AC148
:102FB00002F10BC103F10101A40E046F060E056FAF
:102FC000000E066F000E076F05EC1FF003BF04D064
:102FD00001017F0EDA6F03D00101FF0EDA6F1C8E44
:102FE00011AE32EF19F024C100F125C101F126C163
:102FF00002F127C103F110A405EF18F00401750ECA
:10300000826F29EC0BF00AEF18F00401720E826F48
:1030100029EC0BF004012C0E826F29EC0BF0A3ECD1
:103020001FF0296719EF18F00401200E826F1CEFC2
:1030300018F004012D0E826F29EC0BF030C182F4E0
:103040000401300E822729EC0BF031C182F4040117
:10305000300E822729EC0BF004012E0E826F29EC32
:103060000BF032C182F40401300E822729EC0BF000
:1030700033C182F40401300E822729EC0BF00401E5
:103080006D0E826F29EC0BF004012C0E826F29EC7F
:103090000BF04FC100F150C101F151C102F152C119
:1030A00003F10101A3EC1FF086EC1DF00401480EB2
:1030B000826F29EC0BF004017A0E826F29EC0BF081
:1030C00004012C0E826F29EC0BF066C100F167C180
:1030D00001F168C102F169C103F10101A3EC1FF024
:1030E00086EC1DF00401630E826F29EC0BF00401E5
:1030F0002C0E826F29EC0BF066C100F167C101F163
:1031000068C102F169C103F101010A0E046F000EEA
:10311000056F000E066F000E076F16EC1FF0000E15
:10312000046F120E056F000E066F000E076F36EC6F
:103130001FF0A3EC1FF02AC182F40401300E822795
:1031400029EC0BF02BC182F40401300E822729EC0C
:103150000BF02CC182F40401300E822729EC0BF015
:103160002DC182F40401300E822729EC0BF02EC110
:1031700082F40401300E822729EC0BF02FC182F477
:103180000401300E822729EC0BF030C182F40401D7
:10319000300E822729EC0BF004012E0E826F29ECF1
:1031A0000BF031C182F40401300E822729EC0BF0C0
:1031B00032C182F40401300E822729EC0BF033C1B6
:1031C00082F40401300E822729EC0BF00401730E07
:1031D000826F29EC0BF004012C0E826F29EC0BF0AE
:1031E00000EC20F059C100F15AC101F196EC1AF03F
:1031F0000FB2FEEF18F00FA030EF19F004012C0E03
:10320000826F29EC0BF0200EF86EF76AF66A040163
:103210000900F5CF82F429EC0BF00900F5CF82F418
:1032200029EC0BF00900F5CF82F429EC0BF0090032
:10323000F5CF82F429EC0BF00900F5CF82F429ECEC
:103240000BF00900F5CF82F429EC0BF00900F5CF63
:1032500082F429EC0BF00900F5CF82F429EC0BF095
:1032600033EC0BF00F906CEF19F00401630E826FDA
:1032700029EC0BF004012C0E826F29EC0BF072ECA0
:1032800019F004012C0E826F29EC0BF0E5EC19F01B
:1032900004012C0E826F29EC0BF061EC1AF0040192
:1032A0002C0E826F29EC0BF00101F80E006FCD0E91
:1032B000016F660E026F030E036F87EC19F00401B5
:1032C0002C0E826F29EC0BF077EC1AF033EC0BF03C
:1032D0006CEF19F033EC0BF00301C26B0790109206
:1032E0007BEF1CF0D8900E0EF7EC08F0E8CF00F161
:1032F0000F0EF7EC08F0E8CF01F1100EF7EC08F034
:10330000E8CF02F1110EF7EC08F0E8CF03F101016C
:10331000000E046F000E056F010E066F000E076FA2
:1033200036EC1FF0A3EC1FF02AC182F40401300E2A
:10333000822729EC0BF02BC182F40401300E822786
:1033400029EC0BF02CC182F40401300E822729EC09
:103350000BF02DC182F40401300E822729EC0BF012
:103360002EC182F40401300E822729EC0BF02FC10C
:1033700082F40401300E822729EC0BF030C182F474
:103380000401300E822729EC0BF031C182F40401D4
:10339000300E822729EC0BF004012E0E826F29ECEF
:1033A0000BF032C182F40401300E822729EC0BF0BD
:1033B00033C182F40401300E822729EC0BF00401A2
:1033C0006D0E826F29EC0BF01200120EF7EC08F074
:1033D000E8CF00F1130EF7EC08F0E8CF01F1140E7E
:1033E000F7EC08F0E8CF02F1150EF7EC08F0E8CFA3
:1033F00003F101010A0E046F000E056F000E066F47
:10340000000E076F16EC1FF0000E046F120E056F12
:10341000000E066F000E076F36EC1FF0A3EC1FF0D6
:103420002AC182F40401300E822729EC0BF02BC153
:1034300082F40401300E822729EC0BF02CC182F4B7
:103440000401300E822729EC0BF02DC182F4040117
:10345000300E822729EC0BF02EC182F40401300ECD
:10346000822729EC0BF02FC182F40401300E822751
:1034700029EC0BF030C182F40401300E822729ECD4
:103480000BF004012E0E826F29EC0BF031C182F497
:103490000401300E822729EC0BF032C182F40401C2
:1034A000300E822729EC0BF033C182F40401300E78
:1034B000822729EC0BF00401730E826F29EC0BF0CC
:1034C00012000A0EF7EC08F0E8CF00F10B0EF7EC53
:1034D00008F0E8CF01F10C0EF7EC08F0E8CF02F1AC
:1034E0000D0EF7EC08F0E8CF03F196EF1AF0060E98
:1034F000F7EC08F0E8CF00F1070EF7EC08F0E8CFA2
:1035000001F1080EF7EC08F0E8CF02F1090EF7EC34
:1035100008F0E8CF03F196EF1AF0010100EC20F07B
:10352000078457C100F158C101F107940101E80E69
:10353000046F800E056F000E066F000E076F16EC0D
:103540001FF0000E046F040E056F000E066F000ED4
:10355000076F36EC1FF0880E046F130E056F000E18
:10356000066F000E076F05EC1FF00A0E046F000EC9
:10357000056F000E066F000E076F36EC1FF0A3EC10
:103580001FF001012967CAEF1AF00401200E826FB3
:10359000CDEF1AF004012D0E826F29EC0BF030C133
:1035A00082F40401300E822729EC0BF031C182F441
:1035B0000401300E822729EC0BF032C182F40401A1
:1035C000300E822729EC0BF004012E0E826F29ECBD
:1035D0000BF033C182F40401300E822729EC0BF08A
:1035E0000401430E826F29EC0BF0120087C32AF10D
:1035F00088C32BF189C32CF18AC32DF18BC32EF123
:103600008CC32FF18DC330F18EC331F190C332F1F1
:1036100091C333F10101296B4EEC20F0C5EC1FF092
:103620000101000E046F000E056F010E066F000E03
:10363000076F16EC1FF00E0E0C6E00C10BF0E0ECE5
:1036400008F00F0E0C6E01C10BF0E0EC08F0100E4C
:103650000C6E02C10BF0E0EC08F0110E0C6E03C111
:103660000BF0E0EC08F004017A0E826F29EC0BF00D
:1036700004012C0E826F29EC0BF00401350E826FD1
:1036800029EC0BF004012C0E826F29EC0BF072EC8C
:1036900019F00BEF14F087C32AF188C32BF189C30B
:1036A0002CF18AC32DF18BC32EF18CC32FF18DC366
:1036B00030F18EC331F190C332F191C333F1010186
:1036C000296B4EEC20F0C5EC1FF0880E046F130E32
:1036D000056F000E066F000E076F0AEC1FF0000E5C
:1036E000046F040E056F000E066F000E076F16ECD8
:1036F0001FF00101E80E046F800E056F000E066FCB
:10370000000E076F36EC1FF00A0E0C6E00C10BF0B6
:10371000E0EC08F00B0E0C6E01C10BF0E0EC08F0D1
:103720000C0E0C6E02C10BF0E0EC08F00D0E0C6EEE
:1037300003C10BF0E0EC08F004017A0E826F29EC73
:103740000BF004012C0E826F29EC0BF00401360EF5
:10375000826F29EC0BF004012C0E826F29EC0BF028
:1037600061EC1AF00BEF14F087C32AF188C32BF138
:1037700089C32CF18AC32DF18BC32EF18CC32FF199
:103780008DC330F18FC331F190C332F191C333F166
:1037900001014EEC20F0C5EC1FF0000E046F120E7C
:1037A000056F000E066F000E076F16EC1FF001018B
:1037B0000A0E046F000E056F000E066F000E076FF5
:1037C00036EC1FF0120E0C6E00C10BF0E0EC08F0AE
:1037D000130E0C6E01C10BF0E0EC08F0140E0C6E31
:1037E00002C10BF0E0EC08F0150E0C6E03C10BF0FB
:1037F000E0EC08F004017A0E826F29EC0BF0040172
:103800002C0E826F29EC0BF00401370E826F29EC2D
:103810000BF004012C0E826F29EC0BF0E5EC19F093
:103820000BEF14F087C32AF188C32BF189C32CF165
:103830008AC32DF18BC32EF18CC32FF18DC330F1D0
:103840008EC331F190C332F191C333F10101296B81
:103850004EEC20F0C5EC1FF0880E046F130E056FC0
:10386000000E066F000E076F0AEC1FF0000E046FCB
:10387000040E056F000E066F000E076F16EC1FF0AA
:103880000101E80E046F800E056F000E066F000E3A
:10389000076F36EC1FF0060E0C6E00C10BF0E0EC6B
:1038A00008F0070E0C6E01C10BF0E0EC08F0080EFA
:1038B0000C6E02C10BF0E0EC08F0090E0C6E03C1B7
:1038C0000BF0E0EC08F004017A0E826F29EC0BF0AB
:1038D00004012C0E826F29EC0BF00401380E826F6C
:1038E00029EC0BF004012C0E826F29EC0BF077EC25
:1038F0001AF00BEF14F007A8EEEF1CF00101800E98
:10390000006F1A0E016F060E026F000E036F4BC19F
:1039100004F14CC105F14DC106F14EC107F105ECB2
:103920001FF003BF34EF1DF080EC1DF04BC100F120
:103930004CC101F14DC102F14EC103F1078212ECFD
:103940001EF018C104F119C105F11AC106F11BC11D
:1039500007F1F80E006FCD0E016F660E026F030EB9
:10396000036F05EC1FF00E0E0C6E00C10BF0E0ECC7
:1039700008F00F0E0C6E01C10BF0E0EC08F0100E19
:103980000C6E02C10BF0E0EC08F0110E0C6E03C1DE
:103990000BF0E0EC08F00784010100EC20F057C1C7
:1039A00000F158C101F107940A0E0C6E00C10BF032
:1039B000E0EC08F00B0E0C6E01C10BF0E0EC08F02F
:1039C0000C0E0C6E02C10BF0E0EC08F00D0E0C6E4C
:1039D00003C10BF0E0EC08F034EF1DF007AA34EF60
:1039E0001DF00784010100EC20F057C100F158C11F
:1039F00001F10794060E0C6E00C10BF0E0EC08F02C
:103A0000070E0C6E01C10BF0E0EC08F0080E0C6E16
:103A100002C10BF0E0EC08F0090E0C6E03C10BF0D4
:103A2000E0EC08F0078462C100F163C101F164C1F8
:103A300002F165C103F10794120E0C6E00C10BF088
:103A4000E0EC08F0130E0C6E01C10BF0E0EC08F096
:103A5000140E0C6E02C10BF0E0EC08F0150E0C6EAB
:103A600003C10BF0E0EC08F00798079A04018051BD
:103A700081197F0B0DE09EA8FED714EE00F0815156
:103A80007F0BE126E750812B0F01AD6E36EF1DF065
:103A900076EF0AF018C100F119C101F11AC102F163
:103AA0001BC103F1000E046F000E056F010E066FBF
:103AB000000E076F36EC1FF029A175EF1DF02051A5
:103AC000D8B475EF1DF018C100F119C101F11AC188
:103AD00002F11BC103F1000E046F000E056F0A0E08
:103AE000066F000E076F36EC1FF012000101045143
:103AF000001305510113065102130751031312005D
:103B00000101186B196B1A6B1B6B12002AC182F42E
:103B10000401300E822729EC0BF02BC182F4040142
:103B2000300E822729EC0BF02CC182F40401300EF8
:103B3000822729EC0BF02DC182F40401300E82277C
:103B400029EC0BF02EC182F40401300E822729ECFF
:103B50000BF02FC182F40401300E822729EC0BF008
:103B600030C182F40401300E822729EC0BF031C100
:103B700082F40401300E822729EC0BF032C182F46A
:103B80000401300E822729EC0BF033C182F40401CA
:103B9000300E822729EC0BF012002FC182F40401B1
:103BA000300E822729EC0BF030C182F40401300E74
:103BB000822729EC0BF031C182F40401300E8227F8
:103BC00029EC0BF032C182F40401300E822729EC7B
:103BD0000BF033C182F40401300E822729EC0BF084
:103BE0001200060E1E6E060E1F6E060E206E1E2E94
:103BF000F7EF1DF01F2EF7EF1DF0202EF7EF1DF051
:103C00008B84020E1E6E020E1F6E020E206E1E2E82
:103C100007EF1EF01F2E07EF1EF0202E07EF1EF0FD
:103C20008B9412000101005305E1015303E102539B
:103C300001E1002BD5EC1EF000EC20F03951006FB3
:103C40003A51016F420E046F4B0E056F000E066F66
:103C5000000E076F16EC1FF000C104F101C105F161
:103C600002C106F103C107F118C100F119C101F148
:103C70001AC102F11BC103F107B243EF1EF00AECB7
:103C80001FF045EF1EF005EC1FF000C118F101C157
:103C900019F102C11AF103C11BF1120000EC20F06E
:103CA00059C100F15AC101F1060EF7EC08F0E8CF56
:103CB00004F1070EF7EC08F0E8CF05F1080EF7EC79
:103CC00008F0E8CF06F1090EF7EC08F0E8CF07F1AD
:103CD00005EC1FF000C124F101C125F102C126F15C
:103CE00003C127F1290E046F000E056F000E066F49
:103CF000000E076F16EC1FF0EE0E046F430E056FFB
:103D0000000E066F000E076F0AEC1FF024C104F1CD
:103D100025C105F126C106F127C107F116EC1FF0F8
:103D200000C11CF101C11DF102C11EF103C11FF14F
:103D3000120EF7EC08F0E8CF04F1130EF7EC08F0E0
:103D4000E8CF05F1140EF7EC08F0E8CF06F1150EF8
:103D5000F7EC08F0E8CF07F10D0E006F000E016FD1
:103D6000000E026F000E036F16EC1FF0180E046FAA
:103D7000000E056F000E066F000E076F36EC1FF089
:103D80001CC104F11DC105F11EC106F11FC107F1DF
:103D90000AEC1FF06A0E046F2A0E056F000E066F04
:103DA000000E076F05EC1FF01200BF0EFA6E200E1A
:103DB0003A6F396BD8900037013702370337D8B0E4
:103DC000E6EF1EF03A2FDBEF1EF039073A070353F8
:103DD000D8B412000331070B80093F6F03390F0B72
:103DE000010F396F80EC5FF0406F390580EC5FF0B8
:103DF000405D405F396B3F33D8B0392739333FA935
:103E0000FBEF1EF0405139271200010125EC20F094
:103E1000D8B01200010103510719346FE8EC1FF00C
:103E2000D8900751031934AF800F12000101346B91
:103E30000CEC20F0D8A022EC20F0D8B01200F7EC67
:103E40001FF000EC20F01F0E366F38EC20F00B3521
:103E5000D8B0E8EC1FF0D8A00335D8B01200362F48
:103E600025EF1FF034B10FEC20F012000101346B8C
:103E700004510511061107110008D8A00CEC20F020
:103E8000D8A022EC20F0D8B01200086B096B0A6BA6
:103E90000B6B38EC20F01F0E366F38EC20F007511A
:103EA0000B5DD8A460EF1FF006510A5DD8A460EF47
:103EB0001FF00551095DD8A460EF1FF00451085DA3
:103EC000D8A073EF1FF00451085F0551D8A0053D3D
:103ED000095F0651D8A0063D0A5F0751D8A0073DEB
:103EE0000B5FD8900081362F4DEF1FF034B10FECEF
:103EF00020F0346B0CEC20F0D8903CEC20F0075113
:103F00000B5DD8A490EF1FF006510A5DD8A490EF86
:103F10001FF00551095DD8A490EF1FF00451085D12
:103F2000D8A09FEF1FF0003F9FEF1FF0013F9FEFD2
:103F30001FF0023F9FEF1FF0032BD8B4120034B1E3
:103F40000FEC20F012000101346B0CEC20F0D8B023
:103F5000120041EC20F0200E366F00370137023797
:103F6000033711EE33F00A0E376FE7360A0EE75CBF
:103F7000D8B0E76EE552372FB5EF1FF0362FADEF13
:103F80001FF034B12981D890120001010A0E346F5C
:103F9000200E366F11EE29F03451376F0A0ED8908B
:103FA000E652D8B0E726E732372FD0EF1FF00333C1
:103FB000023301330033362FCAEF1FF0E750FF0FF3
:103FC000D8A00335D8B0120029B10FEC20F01200B0
:103FD000045100270551D8B0053D01270651D8B03E
:103FE000063D02270751D8B0073D032712000051B4
:103FF000086F0151096F02510A6F03510B6F1200D4
:104000000101006B016B026B036B12000101046B79
:10401000056B066B076B12000335D8A01200035125
:10402000800B001F011F021F031F003F1FEF20F026
:10403000013F1FEF20F0023F1FEF20F0032B342B36
:10404000032512000735D8A012000751800B041F6A
:10405000051F061F071F043F35EF20F0053F35EF12
:1040600020F0063F35EF20F0072B342B07251200F8
:104070000037013702370337083709370A370B375C
:1040800012000101296B2A6B2B6B2C6B2D6B2E6B95
:104090002F6B306B316B326B336B120001012A5185
:1040A0000F0B2A6F2B510F0B2B6F2C510F0B2C6FFB
:1040B0002D510F0B2D6F2E510F0B2E6F2F510F0BFC
:1040C0002F6F30510F0B306F31510F0B316F325159
:0C40D0000F0B326F33510F0B336F1200D7
:10BF0000E844F926000C160C2B0C3F0C520C640C68
:10BF1000760C860C960CA50CB30CC10CCF0CDC0C6B
:06BF2000E80CF40C000C1B
:00000001FF
